:100000000C945C000C9492050C94BF050C94840035
:100010000C9484000C9484000C9484000C94840050
:100020000C9484000C9484000C9484000C94840040
:100030000C9484000C9484000C9484000C94840030
:100040000C94EC050C9484000C941E080C94840011
:100050000C9484000C9484000C9484000C94840010
:100060000C9484000C948400000024272A000025AE
:10007000282B000023262904040404040404040299
:100080000202020202030303030303010204081035
:100090002040800102040810200102040810200002
:1000A0000000070002010000030406000000000039
:1000B00000000000F401690411241FBECFEFD4E05A
:1000C000DEBFCDBF11E0A0E0B1E0ECECF1E102C099
:1000D00005900D92AA33B107D9F712E0AAE3B1E077
:1000E00001C01D92A730B107E1F710E0C8EBD0E0E6
:1000F00004C02297FE010E94E008C43BD107C9F763
:100100000E9462040C94E4080C940000FC0110822C
:100110008FEF81831382128282E2848386E9858352
:10012000178216820895EF92FF920F931F93CF9339
:10013000DF93EC019B0177FF03C020E030E005C0B6
:10014000653B710514F024EB30E02983EC806D8170
:1001500070E06E197109882777FD8095982F982F88
:10016000872F762F662730E040E050E00E945B0842
:1001700024EB30E040E050E00E94AF08FF2400E0B4
:1001800010E0102F0F2DFE2CEE24E20EF31E041FA4
:10019000151FC801B70120E430E040E050E00E94A4
:1001A000AF083B832A83DF91CF911F910F91FF907E
:1001B000EF9008955F926F927F928F929F92AF928D
:1001C000BF92CF92DF92EF92FF920F931F93DF9334
:1001D000CF93CDB7DEB76DB67EB6ADB65EB60E9434
:1001E0005C0620913C0130913D0140913E015091CF
:1001F0003F01621773078407950750F02C5E3F4F4D
:100200004F4F5F4F621773078407950708F4AFC01D
:1002100060933C0170933D0180933E0190933F01B8
:10022000E0913A01F0913B01BB2408C082819381A7
:10023000892B09F0B3940680F781E02D3097B1F750
:10024000BB2009F494C08B2D90E0880F991F2DB727
:100250003EB7281B390B0FB6F8943EBF0FBE2DBF1B
:10026000CDB6DEB60894C11CD11CA0913A01B09164
:100270003B0120E013C012968D919C911397892B1E
:1002800049F0E22FF0E0EE0FFF1FEC0DFD1DB183F2
:10029000A0832F5F16960D90BC91A02D109759F753
:1002A0002CC0812F90E07C01EE0CFF1CEC0CFD1C9F
:1002B000D7016D917C91FC013197EE0FFF1FEC0D82
:1002C000FD1D40815181DB0112962D913C911397C8
:1002D000DA0112968D919C9113972817390730F403
:1002E000D7014D935C937183608301E01F5F1B1501
:1002F000C0F2002311F410E011C011E000E0F7CFCC
:10030000E12FF0E0EE0FFF1FEC0DFD1D0190F081DD
:10031000E02D61E080810E9462071F5F1B1580F362
:10032000F6B4EE2400E010E08F2C99241EC0EE2DD0
:10033000F0E0EE0FFF1FEC0DFD1D0190F081E02DB0
:1003400022813381280D391D86B58F1510F4005098
:100350001F4FF82EC8018F0D911D28173907A0F7E0
:1003600060E080810E946207E394EB1400F38A2D21
:10037000952D9C010FB6F8943EBF0FBE2DBF0FB652
:10038000F8947EBE0FBE6DBECF91DF911F910F918D
:10039000FF90EF90DF90CF90BF90AF909F908F90A5
:1003A0007F906F905F9008950F931F938C01FC01D5
:1003B00060838FEF81831382128280913A01909142
:1003C0003B019783868310933B0100933A0160E0E1
:1003D00080810E94620761E0F80180810E944407E9
:1003E00081E01F910F91089580E491E00E948600C2
:1003F00088E491E00E94860080E591E00E948600FA
:100400000895BC0188E491E00E9493000895BC0126
:1004100080E491E00E94930008956BE570E080E431
:1004200091E00E9493006AE570E088E491E00E9408
:1004300093000895EF92FF920F931F930E94DA00AA
:1004400081E791E00E947704882309F4E8C081E7FE
:1004500091E00E947404482F8093640190E074E05E
:10046000959587957A95E1F720915A0130915B0136
:100470008217930709F0D3C050E060E070E020E0FD
:1004800030E081E791E00E947D058091640190E079
:100490008F7090708730910509F482C08830910583
:1004A000C4F48330910509F44DC0843091054CF4B7
:1004B00081309105A9F182309105D4F5892B41F164
:1004C000AEC08530910509F45EC006970CF066C099
:1004D00043C08B30910509F47FC08C30910544F402
:1004E0008930910509F467C00A970CF06DC05CC0B3
:1004F0008D30910509F480C08D3091050CF474C0E5
:100500008E30910509F47AC00F9709F088C07CC03D
:1005100060E080912D010E94620784EB90E00FC0A3
:1005200060E080912D010E94620780E090E011C0A0
:1005300060E080912D010E94620780E090E00E94BF
:1005400001026DC060E080912D010E94620784EB82
:1005500090E00E94070263C084E690E090936E01F1
:1005600080936D0181E090E09093700180936F0122
:100570000E945C066093690170936A0180936B012D
:1005800090936C014CC01092700110926F0160E06A
:1005900070E080911D010E94EC0641C061E001C045
:1005A00060E080911B012DC061E080912B010E94D1
:1005B000620761E006C060E080912B010E94620743
:1005C00060E0809129011DC060E080912D010E94B2
:1005D000620764EB70E01FC060E080912D010E9413
:1005E000620760E070E017C061E080912D010E9419
:1005F00062070E940D0213C061E001C060E08091BB
:100600001F010E9462070BC060E080912D010E94D3
:1006100062076DE570E080E591E00E9493000E9422
:100620005C069B01AC016093650170936601809349
:1006300067019093680180916F019091700101971B
:1006400009F053C08091690190916A01A0916B01FA
:10065000B0916C01281B390B4A0B5B0B80916D012B
:1006600090916E01AA2797FDA095BA2F28173907F8
:100670004A075B07A0F16FEF70E080911D010E94B7
:10068000EC06E0906501F090660100916701109121
:1006900068018091690190916A01A0916B01B0910C
:1006A0006C01A8019701281B390B4A0B5B0B809149
:1006B0006D0190916E01880F991FAA2797FDA09553
:1006C000BA2F281739074A075B0778F0E0926901CB
:1006D000F0926A0100936B0110936C0106C060E018
:1006E00070E080911D010E94EC061F910F91FF9018
:1006F000EF90089540E05BE460E070E081E791E016
:100700000E947A0464E670E080E090E00E946A064D
:1007100060E070E080911D010E94EC0660912F0165
:100720007091300180E491E00E94D4016091310128
:100730007091320188E491E00E94D401609121011E
:100740007091220180E591E00E94D4010E940D0287
:100750006DE570E080E591E00E94930061E080919A
:100760001B010E94440761E080911D010E94440723
:1007700061E080911F010E94440760E08EE00E94CA
:10078000440760E08FE00E94440760E080E10E943F
:10079000440760E081E10E94440761E08EE00E942E
:1007A000620761E08FE00E94620761E080E10E94E1
:1007B000620761E081E10E946207809158010E9416
:1007C000CE06815092403CF081E090E090935D0134
:1007D00080935C0104C010925D0110925C018091D5
:1007E00023010E94CE06815092403CF082E090E0CE
:1007F00090935F0180935E0104C010925F0110929C
:100800005E01809125010E94CE06815092403CF00D
:1008100084E090E0909361018093600104C01092A5
:10082000610110926001809127010E94CE068150E3
:1008300092403CF088E090E09093630180936201E5
:1008400004C0109263011092620180915E01909148
:100850005F0120915C0130915D01820F931F209117
:10086000600130916101820F931F209162013091EC
:100870006301820F931F90935B0180935A0160E0A4
:1008800071E081E791E00E947F0460915A017091CC
:100890005B0181E791E00E946D0560E080911F019E
:1008A0000E94620761E080912D010E94620760E072
:1008B000809129010E94620760E080912B010E94D3
:1008C000620708950E9494060E947A030E941A0209
:1008D000FDCF88E391E090937201809371010895B8
:1008E000862F0E94E60708950E94FF0708950E9440
:1008F000EE070895CB01BA010E94AD0708950F934A
:100900001F93CF93DF938C01EB0109C02196D8018F
:10091000ED91FC910190F081E02DC801099568816D
:100920006623A1F7DF91CF911F910F9108950F9347
:100930001F938C01DC01ED91FC910190F081E02D81
:100940006DE00995D801ED91FC910190F081E02DC9
:100950006AE0C80109951F910F9108952F923F9267
:100960004F925F926F927F928F929F92AF92BF92BF
:10097000CF92DF92EF92FF920F931F93DF93CF936B
:10098000CDB7DEB7A0970FB6F894DEBF0FBECDBFD0
:100990001C016A017B01411551056105710549F48E
:1009A000DC01ED91FC910190F081E02D60E309956F
:1009B00054C0882499245401422E55246624772457
:1009C00001E010E00C0F1D1F080D191DC701B60135
:1009D000A30192010E948D08F80160830894811C94
:1009E000911CA11CB11CC701B601A30192010E9478
:1009F0008D08C901DA016C017D01C114D104E10443
:100A0000F104F1F681E0E82EF12CEC0EFD1EE80C6D
:100A1000F91C3E010894611C711CD501C4010197A9
:100A2000A109B1096C01C818D90814C0F601EE0D6E
:100A3000FF1D60816A3010F4605D01C0695CD10106
:100A4000ED91FC910190F081E02DC1010995089490
:100A5000E108F1086E147F0449F7A0960FB6F894E8
:100A6000DEBF0FBECDBFCF91DF911F910F91FF90E1
:100A7000EF90DF90CF90BF90AF909F908F907F903E
:100A80006F905F904F903F902F900895EF92FF925C
:100A90000F931F93CF93DF93EC017A018B0177FFC4
:100AA0000FC0E881F9810190F081E02D6DE2099598
:100AB00010950095F094E094E11CF11C011D111DAE
:100AC0002AE0B801A701CE010E94AE04DF91CF91C8
:100AD0001F910F91FF90EF9008950F931F938C013A
:100AE000AB01662757FD6095762F0E944605C80129
:100AF0000E9497041F910F910895DC012115310583
:100B000041F4ED91FC910190F081E02D642F099565
:100B100008952A30310519F40E94460508950E946F
:100B2000AE0408951F920F920FB60F9211242F93C7
:100B30003F934F935F936F937F938F939F93AF9365
:100B4000BF93EF93FF938091730190917401892B70
:100B500029F0E0917301F09174010995FF91EF91F3
:100B6000BF91AF919F918F917F916F915F914F91C5
:100B70003F912F910F900FBE0F901F9018951F92CD
:100B80000F920FB60F9211242F933F934F935F93C1
:100B90006F937F938F939F93AF93BF93EF93FF9345
:100BA0008091750190917601892B29F0E091750172
:100BB000F09176010995FF91EF91BF91AF919F91CF
:100BC0008F917F916F915F914F913F912F910F90F6
:100BD0000FBE0F901F9018951F920F920FB60F9295
:100BE00011242F938F939F93AF93BF93809177019D
:100BF00090917801A0917901B0917A010196A11D9F
:100C0000B11D8093770190937801A0937901B093FF
:100C10007A0180917B0190917C01A0917D01B0913E
:100C20007E018050904CAF4FBF4F80937B019093DB
:100C30007C01A0937D01B0937E0127C080917B0150
:100C400090917C01A0917D01B0917E0180589E43DE
:100C5000A040B04080937B0190937C01A0937D01E4
:100C6000B0937E0180917F0190918001A0918101DC
:100C7000B09182010196A11DB11D80937F019093D7
:100C80008001A0938101B093820180917B019091BA
:100C90007C01A0917D01B0917E0181589E43A040CE
:100CA000B04060F6BF91AF919F918F912F910F90BF
:100CB0000FBE0F901F9018958FB7F89420917F0169
:100CC0003091800140918101509182018FBFB90123
:100CD000CA010895EF92FF920F931F937B018C013D
:100CE0008FB7F89440917F0150918001609181010C
:100CF000709182018FBF2FB7F89480917F019091FE
:100D00008001A0918101B09182012FBF841B950BBE
:100D1000A60BB70BE816F9060A071B0760F71F9129
:100D20000F91FF90EF900895789484B5826084BD10
:100D300084B5816084BD85B5826085BD85B58160DF
:100D400085BDEEE6F0E0808181608083E1E8F0E03F
:100D5000808182608083808181608083E0E8F0E030
:100D6000808181608083E1EBF0E08081846080831A
:100D7000E0EBF0E0808181608083EAE7F0E0808151
:100D800084608083808182608083808181608083B1
:100D90008081806880831092C10008958F70909147
:100DA00033019295990F990F907C982B90937C002A
:100DB00080917A00806480937A0080917A0086FD29
:100DC000FCCF2091780040917900942F80E030E0B2
:100DD000282B392BC90108951F93CF93DF93182F28
:100DE000EB0161E00E944407E12FF0E0E156FF4F84
:100DF0008491833051F480918000806880938000DA
:100E0000D0938900C09388003BC0843051F4809116
:100E10008000806280938000D0938B00C0938A0012
:100E20002FC0813039F4209729F184B5806884BDC2
:100E3000C7BD26C0823039F42097E1F084B58062C6
:100E400084BDC8BD1DC0863041F48091B00080686B
:100E50008093B000C093B30013C0873041F48091F9
:100E6000B00080628093B000C093B40009C0C03865
:100E7000D10514F460E001C061E0812F0E94620797
:100E8000DF91CF911F910895282F30E0C901855738
:100E90009F4FFC01949129583F4FF9018491882379
:100EA00081F0E82FF0E0E859FF4FE491F0E066238D
:100EB00029F4808190958923808308958081892BEE
:100EC00080830895482F50E0CA0181569F4FFC014E
:100ED0002491CA0185579F4FFC01949149585F4F57
:100EE000FA0134913323C1F1222331F1233021F46B
:100EF000809180008F7705C0243031F4809180008C
:100F00008F7D8093800018C0213019F484B58F77CD
:100F100004C0223021F484B58F7D84BD0DC02630FD
:100F200021F48091B0008F7705C0273029F480919B
:100F3000B0008F7D8093B000E32FF0E0E359FF4FC6
:100F4000E491F0E0662329F48081909589238083E1
:100F500008958081892B80830895EF92FF920F93EB
:100F60001F937B018C0122E030E040E050E00E94C2
:100F7000AF08205C3D4B404F5F4FCA01B901A8014B
:100F800097010E94AF08C901DA010197A109B109CF
:100F9000292F3A2F4B2F552747FD5A950196A11D12
:100FA000B11D2093C50081508093C400E1ECF0E0B6
:100FB0008081806180838081886080838081806877
:100FC00080831F910F91FF90EF900895982F80914B
:100FD000C00085FFFCCF9093C600089580918301E7
:100FE0009091840180589F4F209185013091860116
:100FF000821B930B60E870E00E947A08089540918C
:10100000850150918601809183019091840184171C
:10101000950719F42FEF3FEF0FC0FA01E957FE4F84
:101020002081CA01019660E870E00E947A089093DE
:1010300086018093850130E0C90108951F920F92C7
:101040000FB60F9211242F933F934F935F936F939B
:101050007F938F939F93AF93BF93EF93FF934091B1
:10106000C600E0918301F0918401CF01019660E810
:1010700070E00E947A089C01809185019091860120
:101080002817390739F0E957FE4F40833093840120
:1010900020938301FF91EF91BF91AF919F918F9129
:1010A0007F916F915F914F913F912F910F900FBE64
:1010B0000F901F901895629FD001739FF001829F3F
:1010C000E00DF11D649FE00DF11D929FF00D839FD7
:1010D000F00D749FF00D659FF00D9927729FB00D74
:1010E000E11DF91F639FB00DE11DF91FBD01CF0187
:1010F0001124089597FB092E07260AD077FD04D006
:1011000049D006D000201AF4709561957F4F08955C
:10111000F6F7909581959F4F0895A1E21A2EAA1B8C
:10112000BB1BFD010DC0AA1FBB1FEE1FFF1FA21797
:10113000B307E407F50720F0A21BB30BE40BF50B94
:10114000661F771F881F991F1A9469F7609570951D
:10115000809590959B01AC01BD01CF01089597FB4F
:10116000092E05260ED057FD04D0D7DF0AD0001C6B
:1011700038F450954095309521953F4F4F4F5F4F34
:101180000895F6F790958095709561957F4F8F4FF4
:101190009F4F0895AA1BBB1B51E107C0AA1FBB1F8D
:1011A000A617B70710F0A61BB70B881F991F5A95F3
:1011B000A9F780959095BC01CD010895EE0FFF1F12
:0C11C0000590F491E02D0994F894FFCF05
:1011CC00486F6C612C20736F7920656C20726F6294
:1011DC006F74206E756D65726F200008000B000433
:1011EC0000020001000200030003000500070009D3
:0A11FC00000A00010000000070046A
:00000001FF
